:100000000C9432040C9479040C9479040C947904C3
:100010000C9479040C9479040C9479040C9479046C
:100020000C9479040C9479040C94982F0C946A30F5
:100030000C941A2A0C9479040C9479040C94790485
:100040000C9479040C9479040C9479040C9479043C
:100050000C9479040C94732A0C9479040C9479040C
:100060000C9479040C9479040C9479040C9479041C
:100070000C9479040C9479040C9479040C9479040C
:100080000C9479040C9479040C9479040C947904FC
:100090000C9479040C9479040C9479040C947904EC
:1000A0000C9479040C9479040C9479048F056E05F2
:1000B000700572057405760578057A057C057E0560
:1000C00001170417251736173E1749174C174F17F6
:1000D000521798179817551758175D176A177717FB
:1000E0007A177E178B17C61FC61FF81FF81F4520EB
:1000F0006320842184216E20032114211421742182
:10010000842184217D2124222422362236222D227C
:100110003622362236222422242232223622362247
:100120003222D730FE30F631FE30F6314A316D31B1
:10013000F631C431D331165C1E001F0020002100AF
:100140002200230024002500260027002D002E0079
:100150002A0053005400550056002B0014001A00CA
:100160000800150017001C0018000C0012001300F6
:100170002F0030004C005F00600061006700390014
:1001800004001600070009000A000B000D000E0015
:100190000F0033003400310028005C005D005E0079
:1001A0005700E10064001D001B0006001900050057
:1001B00011001000360037003800E50052005900E9
:1001C0005A005B002A00E000E300E20000000000AB
:1001D00000002C00000000000000E600015150006B
:1001E00051004F0062006300580035003A003B00A8
:1001F0003C003D003E003F00400041004200430003
:10020000440045000100010001000100010001005F
:100210000100520001000100010001000100010085
:10022000010001000100005C01000100010001006B
:1002300001000100500051004F00010001000100C9
:1002400001000100010001000100010001000100A6
:100250000100010001000100010001000100010096
:100260000100010001000100010001000100010086
:1002700001000100010001000100A900AA00A8007E
:10028000000000000000010000000000000001006C
:100290000100010001000100010001000100010056
:1002A0000100010001000100010001000100010046
:1002B0000100010001000100010001000100010036
:1002C0000100010001000100010001000100010026
:1002D0000100010001000100010001000100010016
:1002E0000100010001000100010001000100010006
:1002F00001000100010001000100010001000100F6
:1003000001000100010001000100010001000100E5
:1003100001000100010001000100010001000100D5
:1003200001000100010001000100010001000100C5
:1003300001000100000000000000010000000000BA
:1003400000000100010001000100010001000100A6
:100350000100010001000100010001000100010095
:100360000100010001000100010001000100010085
:100370000100010001000100010001000100010075
:100380000100010001000100010001000100010065
:100390000100010001000100010001000100010055
:1003A0000100010001000100010001000100010045
:1003B0000100010001000100010001000100010035
:1003C0000100010001000100010001000100010025
:1003D0000100010001000100010001000100010015
:1003E0000100010001000100000000000000010008
:1003F00000000000000001000100010001000100F8
:1004000001000100010000000000000000002A2B94
:1004100028000000000000000000000000000000B4
:100420000029000000002C1E34202122243426271D
:10043000252E362D3738271E1F202122232425263E
:100440003333362E37381F0405060708090A0B0C0C
:100450000D0E0F101112131415161718191A1B1C54
:100460001D2F3130232D350405060708090A0B0C12
:100470000D0E0F101112131415161718191A1B1C34
:100480001D2F3130354C000000000000000000003E
:10049000000000000000000000000000000000005C
:1004A000000000000000000000007E0F00D4FFFFED
:1004B000FFC7000000781E0F0500047F3F1F643255
:1004C00014643214783C1E1E140A052223252628A3
:1004D000292A2C2D2F3032333536383A3B3D3E40D9
:1004E00042434547494A4C4E5051535557595A5C1F
:1004F0005E6062646668696B6D6F71737577797B36
:100500007D7F81838587898A8C8E90929496989A34
:100510009C9E9FA1A3A5A7A8AAACAEAFB1B3B4B649
:10052000B8B9BBBCBEBFC1C2C3C5C6C7C9CACBCCA4
:10053000CDCED0D1D2D2D3D4D5D6D7D7D8D9D9DA77
:10054000DADBDBDBDCDCDCDCDCDDDDDDDDDCDCDCEC
:10055000DCDCDBDBDBDADAD9D9D8D7D7D6D5D4D314
:10056000D2D2D1D0CECDCCCBCAC9C7C6C5C3C2C1E9
:10057000BFBEBCBBB9B8B6B4B3B1AFAEACAAA8A746
:10058000A5A3A19F9E9C9A98969492908E8C8A89FE
:10059000878583817F7D7B79777573716F6D6B69DB
:1005A00068666462605E5C5A5957555351504E4CB0
:1005B0004A4947454342403E3D3B3A38363533325F
:1005C000302F2D2C2A292826252322FFAA7F5540AB
:1005D0000001020304060708090A0B0C0D0E0500B2
:1005E00001010101010101010102020202020202F4
:1005F00002020303030303030303040404040404C7
:10060000040505050505060606060607070707078C
:1006100008080808090909090A0A0A0B0B0B0C0C3F
:100620000C0D0D0D0E0E0E0F0F0F101011111112DB
:100630001213131414151516161717181819191A5A
:100640001A1B1B1C1D1D1E1E1F20202122222324BD
:1006500024252626272829292A2B2C2D2D2E2F30FC
:10066000313232333435363738393A3B3C3D3E3F10
:10067000404142434445464748494A4C4D4E4F50FD
:10068000515354555658595A5B5D5E5F61626465BB
:100690006668696B6C6D6F7072737577787A7B7D45
:1006A0007E8082838587888A8C8E8F919395969899
:1006B0009A9C9EA0A2A3A5A7A9ABADAFB1B3B5B7B5
:1006C000BABCBEC0C2C4C6C9CBCDCFD1D4D6D8DB8C
:1006D000DDDFE2E4E7E9EBEEF0F3F5F8FAFDFF1E0B
:1006E000034200610072006C006500790063006FD6
:1006F0000072006E00200053004D00440000001402
:10070000035000330044002000530074006F007257
:1007100000650000000403090409025B00030100F6
:10072000A0C8090400000103010100092111010012
:10073000012240000705810308000A0904010002A4
:100740000300000009211101000122220007058297
:100750000320000107050303200001090402000132
:1007600003000000092111010001227B000705841C
:100770000320000A120110010000000833704947ED
:100780000100010200010660FF0961A10109621573
:100790000026FF009520750881020963150026FFD9
:1007A00000952075089102C005010902A10185028A
:1007B0000901A1000509190129081500250195085D
:1007C000750181020501093009311581257F9502E6
:1007D0007508810609381581257F95017508810600
:1007E000050C0A38021581257F950175088106C020
:1007F000C005010980A101850319012AB70015016F
:1008000026B700950175108100C0050C0901A101F2
:10081000850419012AA002150126A0029501751070
:100820008100C005010906A101050719E029E715A6
:100830000025019508750181029501750881010562
:1008400007190029FF150026FF009506750881008D
:100850000508190129059505750191029501750392
:100860009101C00011241FBECFEFDAE0DEBFCDBF83
:1008700004B603FE27C08091730390917403A09186
:100880007503B09176038730904BA740B04BD1F4FD
:1008900010927303109274031092750310927603F2
:1008A00014BE84B7877F84BF0FB6F894A895809153
:1008B0006000886180936000109260000FBEE0E0ED
:1008C000F8E3099511E0A0E0B1E0ECE3F7E602C03F
:1008D00005900D92A03EB107D9F723E0A0EEB1E05C
:1008E00001C01D92A337B207E1F70E94592C0C9466
:1008F0009C330C9400000F931F93CF93DF9300D091
:10090000CDB7DEB70E944D1BAEE3B1E041E050E051
:100910008D91E82FE295EF70F0E021A18F70BA0180
:1009200002C0660F771F8A95E2F7CB01962F90954C
:10093000922391A392A1892B82A371E0A334B707DC
:1009400039F78FEF898383E08A8304E110E022E0A6
:1009500030E0AE014F5F5F4F60E080E40E94241CF6
:1009600022E030E0AE014F5F5F4F6CE080E40E9418
:10097000241CACE2B1E080E061E070E0883098F4E3
:100980009C91E92FE295EF70F0E041A19F709B01EF
:1009900001C0220F9A95EAF7922F9095942391A384
:1009A00092A1292B22A38F5F1196823139F78FEF05
:1009B00090E722E0815090402040E1F700C0000025
:1009C0000F900F90DF91CF911F910F9108952F926B
:1009D0003F924F925F926F927F928F929F92AF92CF
:1009E000BF92CF92DF92EF92FF920F931F93CF931C
:1009F000DF93CDB7DEB760970FB6F894DEBF0FBEBA
:100A0000CDBF0EE311E01C830B836C014C0114E19C
:100A1000810E911CA12CDE82CD82D6018D919D91FB
:100A20000D90BC91A02D8F839887A987BA87F60176
:100A30001082118212821382AB81BC818D91BC83A2
:100A4000AB83E82EE2949FE0E922F12CF70191A11B
:100A50008F7022242394312C01C0220C8A95EAF74E
:100A6000892F822981A382A1B22CB0948B2182A3E9
:100A70000E94640A04E110E022E030E0AE014F5F22
:100A80005F4F62E180E40E94511C8981082F017050
:100A90000B87182F12701C87182F1470082F0870DE
:100AA000282F20712D87382F30723E87982F907411
:100AB0009F8780789A81A92FA170A88B9270ACE251
:100AC000B1E020E030E0422F50E0FA013897EA3000
:100AD000F105B0F4EA5AFF4F0C948E324C8520C0D9
:100AE000412F1EC0402F1CC04D851AC04E8518C016
:100AF0004F8516C0482F14C0488912C0492F10C016
:100B00006C91E62FE295EF70F0E040A150E06F703D
:100B100002C0559547956A95E2F7417001C04B8533
:100B2000F601408051806280738041110DC041E028
:100B300050E060E070E0022E04C0440F551F661FB5
:100B4000771F0A94D2F703C040E050E0BA0144296D
:100B5000552966297729F60140835183628373837F
:100B60002F5F3F4F11962231310509F0ACCFD701ED
:100B700091968C919197B8229196BC92919792966A
:100B80008C919297822992968C93B4E0CB0ED11CD3
:100B900081E0ED81FE8140815181628173810F810D
:100BA000188529853A85401751076207730709F4AC
:100BB00080E0A82AC814D90409F02DCF8A2D6096A8
:100BC0000FB6F894DEBF0FBECDBFDF91CF911F915E
:100BD0000F91FF90EF90DF90CF90BF90AF909F90DC
:100BE0008F907F906F905F904F903F902F900895DF
:100BF00081E0089581E008950C94FA0508950C941D
:100C0000FE051F93CF93DF9300D000D01F92CDB786
:100C1000DEB749835A836B833091700289819A8150
:100C2000311114C0662359F0222349F00E945D2738
:100C3000182F682F89819A810E94062703C00E947D
:100C40003127182F69817A81812F04C00E945D2786
:100C500069817A810F900F900F900F900F90DF9124
:100C6000CF911F910C946A18FC01262F408151816D
:100C70006281738184810C940106CF93DF93EC0130
:100C800060E00E943406BE01DF91CF910C94FF0515
:100C90008F929F92AF92BF92CF92DF92EF92FF928C
:100CA0000F931F936B017C0181E090E0A0E0B0E026
:100CB0004C015D0104C0880C991CAA1CBB1C4A9500
:100CC000D2F7AC01BD0104C0440F551F661F771F4A
:100CD0002A95D2F7482959296A297B2904C0880F07
:100CE000991FAA1FBB1F0A95D2F78A019B010C21ED
:100CF0001D212E213F21401751076207730739F448
:100D0000BC01CD016C297D298E299F290AC08095BF
:100D10009095A095B095BC01CD016C217D218E21CF
:100D20009F211F910F91FF90EF90DF90CF90BF9088
:100D3000AF909F908F9008950F93382F262F60913A
:100D4000E5027091E6028091E7029091E802042F9B
:100D5000432F0E9448060F910C9442260E94330AAA
:100D60000E940F080C946F0A0C946B0A08950E945D
:100D700012220E94B6062FEF84E39CE021508040AF
:100D80009040E1F700C000000C94992A0F931F9344
:100D9000CF93DF938C0161E00E943406EC01B8012F
:100DA0000E945916882309F44BC0B801CE010E9455
:100DB000FC05882309F444C0B801CE010E949F19A4
:100DC0008823F1F1B801CE010E94F1198823C1F105
:100DD000B801CE010E941C1B882391F1B801CE01FD
:100DE0000E940215882361F1F8018281882309F1AC
:100DF000CA358DE5D807C1F050F4C115FCE5DF0711
:100E000081F0CE3DDC45A9F40E946E2919C0CB3596
:100E1000EDE5DE0761F0CC35DD4559F40E94F027A1
:100E200008C00E94B7060CC00E94F92702C00E94A9
:100E3000FC27C801DF91CF911F910F910C94F80509
:100E400080E0DF91CF911F910F910895DF92EF9293
:100E5000FF920F931F93CF93DF93E82FF0E0EA5FA9
:100E6000FB4FD490282F26952695269530E0F90142
:100E7000EA55FB4F0491877010E0082E02C01595CB
:100E800007950A94E2F701701127F901EA56FB4F22
:100E9000E490F12C082E02C0F594E7940A94E2F74E
:100EA00091E0E922FF24F901EA57FB4FC491D0E019
:100EB00002C0D595C7958A95E2F7C170DD27011567
:100EC000110519F081EE0E94531EE114F10419F08E
:100ED00086EE0E94531E8D2D0E947C1FEF2819F074
:100EE00086EE0E94FD1E012B19F081EE0E94FD1E70
:100EF000CD2B51F08CE2DF91CF911F910F91FF909C
:100F0000EF90DF900C947C1FDF91CF911F910F9198
:100F1000FF90EF90DF900895EF92FF920F931F9351
:100F2000CF93DF93EC01162F0AE08881882309F420
:100F300055C0813009F043C08981813041F47E0180
:100F400082E0E80EF11C8A810E947C1F09C0823079
:100F500049F47E01E2E0EE0EF11C8A810E94531EEC
:100F6000E7012FC0833041F47E01F2E0EF0EF11C67
:100F70008A810E94FD1EF4CF843011F0219621C099
:100F80002A81229680E090E030E0205331092A3017
:100F9000310558F4089FA001099F500D1124C90183
:100FA000840F951F21962881EFCF009751F0EFE92C
:100FB000FFE03197F1F700C000000197F6CF0E94E3
:100FC00026072196812F882309F4AFCFEFE9FFE0B0
:100FD0003197F1F700C000008150F5CFDF91CF913C
:100FE0001F910F91FF90EF90089560E00C948C0793
:100FF00008950C94F80781E00895CF93C82F0E94BC
:10100000FB07882351F0C0FF02C02B9A01C02B9828
:10101000C1FF02C02A9A01C02A98CF910895239A4D
:101020002B98229A2A980895CF93C82F0E94F907E7
:101030008C2F0E94FD07CF91089580E090E00895E5
:101040000895880F991FFC01EA54FB4F85919491F4
:101050000895CF93DF930E946A180E944109EC0122
:101060008115904508F041C0C11580E4D80708F00B
:10107000D1C0C83ED10510F5C03ED10508F0FDC075
:10108000C83AD10578F4C53AD10508F0A2C0C130FC
:10109000D10509F4F2C008F4EEC0C430D10508F05F
:1010A000ECC0E9C0CF3BD10508F49BC0C03CD105E2
:1010B00008F4E1C0CE01805C91099EC0C11590E2A8
:1010C000D90758F4C11521E0D20708F0D6C0C03FB7
:1010D000D10508F4D0C0D065D0C0C11580E3D807D1
:1010E00008F08EC0CE019F7087C0C11595E5D90765
:1010F00008F043C0C11524E5D20708F0A2C0C1150D
:1011000082E5D80708F5C11591E5D90708F085C033
:10111000CE0174E0969587957A95E1F783709C2FC0
:10112000937021E030E002C0220F331F9A95E2F75E
:101130003C68382BCF70C695C69580E2C89FE00109
:101140001124C22BD32B99C09E01237033278C2FDF
:1011500086958695C115D34508F064C0C1E0D0E0FE
:1011600002C0CC0FDD1F2A95E2F720E2829FC0016A
:101170001124C82BD92BDC6880C0C11529E5D20702
:10118000A0F4C11588E5D80708F060C0C11596E540
:10119000D90708F070C08C2F0E94D5098F71C82F15
:1011A000D0E0DC2FCC27D06268C0C1152AE5D20779
:1011B00008F451C0CE0190568115904208F05BC0F2
:1011C0008D2F8F710E94D509DD27D0628F71D82BAA
:1011D00054C0C55AD0E0CF58DE4FC881D0E0D064AB
:1011E0004CC0C85AD0E0CC0FDD1FCD5BDE4F09905C
:1011F000D881C02DD46441C00E942108EC013DC0BB
:10120000CE019927D3FF03C0EC01D86C36C0EC01A6
:10121000D06C33C0DF70D06A30C0DC2FCC27C16FF8
:10122000D06A2BC0C1E0D0E002C0CC0FDD1F2A95F0
:10123000E2F720E2829FC0011124C82BD92BDA6883
:101240001CC0DC2FCC27C46FD06A17C0DC2FCC2782
:10125000C06FD06A12C08C2F8F700E94D50994E0A5
:10126000D695C7959A95E1F7CF70D0E0DC2FCC27C3
:10127000D069C82B02C0C0E0D0E0CE01DF91CF9191
:1012800008958238910569F1B0F48133910509F42C
:101290006DC048F48932910509F463C08A32910522
:1012A00009F469C008958533910509F455C089335F
:1012B0009105B9F00895833E910569F138F4803EB7
:1012C0009105B1F0823E910509F10895863E9105A0
:1012D000A9F1873E9105B9F1843E910509F064C0FA
:1012E00023C02091060320FD4FC021FD4DC008956D
:1012F0008091060380FD44C08091070380FF44C0B5
:101300008091060384FD42C083EE4DC080910603A8
:1013100082FF38C0F5CF8091060382FD33C08091F3
:10132000070380FD31C0ECCF8091070381FF32C0FD
:101330008091060384FD2AC087EE35C080910603A4
:1013400083FF26C0F5CF8091060383FD21C08091E5
:10135000070381FD1FC0ECCF8091060385FD1CC0F3
:101360001DC08091060385FD19C016C0809106033B
:1013700086FD16C017C08091060386FD13C010C0FD
:1013800089E311C082EE0FC080EE0DC080E00BC07B
:1013900086EE09C084EE07C089E205C085E303C07C
:1013A0008AE201C081E390E008959091060392FFE4
:1013B0000DC0282F2871283019F4877F846006C05B
:1013C000282F2471243011F48B7F886093FF0DC087
:1013D000282F2871283119F4877E846106C0282FB0
:1013E0002471243111F48B7E88612091070320FF42
:1013F0000DC0382F3871383019F4877F816006C0EE
:10140000382F3171313011F48E7F886021FF0DC08B
:10141000282F2871283119F4877E816106C0282F72
:101420002171213111F48E7E886194FD877E0895AB
:101430000C9433160E94880A2FEF86E791E0215022
:1014400080409040E1F700C000000E94880A80E0E0
:101450000E94570A60FF04C00E94180A0C94992A3F
:1014600008950C941A0A0E94C628811102C00E9495
:101470006E290E94D1288093FA020E94D928909365
:101480000703809306030E94310A0E94D528682F23
:1014900070E080E090E00E9408266091E502709183
:1014A000E6028091E7029091E8020C94402624E045
:1014B000829FC0011124FC01E45EFC4F60817181B8
:1014C000828193810895089580EA8A95F1F70895BD
:1014D00008950C94680A0C94690A0C94680A0C9498
:1014E0006D0A0E947B04E8E0F3E0ACE1B3E0119206
:1014F0001192119211921D921D921D921D9283E0E4
:10150000EC31F807A1F785E00E949B0A0C94AE0627
:10151000CF9388E093E00E94E704C82F282F45E08E
:101520006CE173E088E093E00E949C0A0E94B4069C
:101530008C2FCF9108950895FF920F931F93CF930F
:10154000DF93F82ED92F8B01C42F222349F081E09D
:101550008093E4010E944C2A9093E3018093E2017E
:101560008091E4018823F1F08091E2019091E30100
:101570000E94642A0697B0F0EF2DFD2FD80180E07D
:1015800090E04C2F50E08417950754F4019111918D
:10159000219131910D931D932D933D930196F3CF9E
:1015A0001092E401DF91CF911F910F91FF90089568
:1015B0008091EB0180FF0BC06091090185E0689F7D
:1015C000B001112475956795759567952BC081FFBE
:1015D00009C06091090185E0689FB00111247595EB
:1015E000679520C082FF07C06091090185E0689F70
:1015F000B001112417C09091EA019923D1F06091B4
:101600000801961788F72091090185E0289F90012D
:101610001124929FA001939F500D112470E0CA01E4
:101620000E9458326038710540F46115710519F453
:1016300006C065E070E0862F08958FE7089581E089
:1016400008958091EB0180FF08C06091050170E072
:10165000759567957595679521C081FF06C0609166
:10166000050170E07595679519C082FF04C060910F
:10167000050170E010C09091E901992399F0609103
:1016800004019617A0F780910501899FC0011124DC
:1016900070E00E9458326038710540F461157105A0
:1016A00019F406C061E070E0862F08958FE7089571
:1016B00081E00895803F21F40E94D80A819504C0FA
:1016C000813F29F40E94D80A8093EF010895823F58
:1016D00021F40E94D80A819504C0833F29F40E9416
:1016E000D80A8093EE010895893F19F40E94210BD6
:1016F00005C08A3F31F40E94210B81958093F0014F
:1017000008958B3F21F40E94210B819504C08C3FEA
:1017100029F40E94210B8093F10108959CE0980F19
:10172000953078F421E030E0A90102C0440F551F44
:101730009A95E2F7CA019091ED01892B8093ED0112
:1017400008958D3F21F48091EB0181600BC08E3FA5
:1017500021F48091EB01826005C08F3F29F48091D4
:10176000EB0184608093EB010895803F39F4909100
:10177000EF0197FF35C01092EF0159C0813F29F466
:101780009091EF011916BCF32BC09091EE01823FAE
:1017900029F497FF25C01092EE0149C0833F19F448
:1017A0001916CCF31DC09091F001893F29F4191648
:1017B000BCF41092F0013BC08A3F19F497FF10C0AF
:1017C000F8CF8B3F39F49091F10197FF09C0109247
:1017D000F1012DC08C3F21F49091F1011916BCF359
:1017E0009CE0980F953080F421E030E0A90102C020
:1017F000440F551F9A95E2F7CA0180959091ED012B
:1018000089238093ED0113C08D3F21F48091EB017A
:101810008E7F0BC08E3F21F48091EB018D7F05C040
:101820008F3F29F48091EB018B7F8093EB018091B6
:10183000EE01811106C08091EF01811102C010926A
:10184000EA018091F001811106C08091F1018111BE
:1018500002C01092E90108950E944C2A2091EE01E5
:10186000211104C02091EF01222321F09093E8017F
:101870008093E7012091F001211104C02091F10132
:10188000222321F09093E6018093E5018CEE91E014
:101890000C94B91CEF92FF920F931F93CF93DF9399
:1018A00000D000D000D0CDB7DEB786E0ECEEF1E09E
:1018B000DE01119601900D928A95E1F7E090EE011C
:1018C000F090EF010091F0011091F1011092EE0102
:1018D0001092EF011092F0011092F101E11003C09B
:1018E000FF2009F45DC08091E7019091E8010E941A
:1018F000642AAC019091EA01992339F020910A0100
:1019000030E02417350758F04BC020910B018AE0D6
:10191000289F900111242417350718F041C09F3FDC
:1019200019F09F5F9093EA01EE2061F00E94D80ABF
:101930001E1414F09FEF01C091E0989F902D112488
:101940009093EE01FF2061F00E94D80A1F1414F05A
:101950009FEF01C091E0989F902D11249093EF018B
:101960003091EE013323E1F02091EF012223C1F009
:1019700045EB3403C0011124992319F09093EE0133
:1019800003C081E08093EE0135EB2303C0011124F5
:10199000992319F09093EF0103C081E08093EF0148
:1019A000011103C0112309F45DC08091E5019091FC
:1019B000E6010E94642AAC019091E901992339F073
:1019C0002091060130E02417350758F04BC02091D4
:1019D00007018AE0289F900111242417350718F089
:1019E00041C09F3F19F09F5F9093E901002361F090
:1019F0000E94210B101614F09FEF01C091E0989FF8
:101A0000902D11249093F001112361F00E94210B7D
:101A1000111614F09FEF01C091E0989F902D1124B2
:101A20009093F1013091F0013323E1F02091F10125
:101A30002223C1F045EB3403C0011124992319F08E
:101A40009093F00103C081E08093F00135EB230314
:101A5000C0011124992319F09093F10103C081E092
:101A60008093F1018091EE0181110BC08091EF0113
:101A7000811107C08091F001811103C08091F101B3
:101A800081110E942C0CEB82FC820D831E8386E068
:101A9000FE013196ACEEB1E001900D928A95E1F72E
:101AA00026960FB6F894DEBF0FBECDBFDF91CF9163
:101AB0001F910F91FF90EF900895ECEEF1E086E01A
:101AC000DF011D928A95E9F71092EA011092E9016F
:101AD0001092EB010895EF92FF920F931F93CF9313
:101AE000DF938B01682F11110AC0442329F0E82FDE
:101AF000F0E0E152FA4F6491762F862F75C0212FC6
:101B000030E0E82FF0E0442321F0E152FA4FE49175
:101B1000F0E046E0049FC0011124CFEFD0E0BE0109
:101B20000E9444324BEA4603C001479F900D1124A6
:101B3000800F911D800F911D982F990F890FAE0175
:101B4000421B530B4E9FD0014F9FB00D5E9FB00DB7
:101B500011249B2F189FA0011124452F55278E017A
:101B6000041B150B0E9FA0010F9F500D1E9F500DC3
:101B700011247E01E81AF108E29E8001E39E100D17
:101B8000F29E100D1124212F3327C21BD30BCE9FA1
:101B90009001CF9F300DDE9F300D11246230710512
:101BA000A9F048F46115710569F061307105C9F457
:101BB0008B2F752F0DC06430710581F058F06630A1
:101BC000710579F47E2F8B2F932F0DC0832F7B2FE0
:101BD0009E2F09C08E2F7B2F952F05C08E2F732F20
:101BE00002C07E2F852F692FDF91CF911F910F911A
:101BF000FF90EF90089541E00E946B0D08950895C5
:101C00000E94FB0D0895CF93DF93762FE901682F93
:101C1000842F0E94000E798368838A83DF91CF919D
:101C2000089580913003282F269530E02115310545
:101C300019F48170826005C02B32310524F0817067
:101C4000846580933003089588E090E00C943D33E0
:101C5000CF92DF92EF92FF926B017C010E94110EF6
:101C6000B701A60188E090E0FF90EF90DF90CF9061
:101C70000C945B3360913003709131038091320397
:101C8000909133030C94280EE0E3F3E083E080832B
:101C900011828FEF828383831482608171818281BC
:101CA00093810C94280E8091300380FF02C08695AA
:101CB000089580E0089590913403933018F49F5F65
:101CC00090933403882351F0609130037091310375
:101CD00080913203909133030C94280E089581E093
:101CE0000C945B0E90913403992319F091509093CA
:101CF0003403882351F06091300370913103809157
:101D00003203909133030C94280E089581E00C94D3
:101D1000720E80913403089580933403662351F04A
:101D200060913003709131038091320390913303BD
:101D30000C94280E089560E00C948C0E8091310371
:101D4000089580913203089580913303089570E0DF
:101D50000C94D115CF92DF92EF920F931F93CF93F4
:101D6000DF93CDB7DEB7AD970FB6F894DEBF0FBEE9
:101D7000CDBF609110018091300380FF0AC0E0ED7B
:101D8000F5E0AE014F5F5F4F8E01025D1F4FCA014C
:101D900014C08091110190911201891780F7E82FEA
:101DA000F0E09F01220F331FE20FF31FEB5CFC4FAB
:101DB0001182108212828F5FF0CF249130E0D9011E
:101DC000AA0FBB1F2A0F3B1FD901AB5CBC4FCD90A4
:101DD000DD90EC90DA01CD92DD92ED92AD0131967D
:101DE000A017B10751F720910F01B3E02B9F800D91
:101DF000911D11240E94A70EAD960FB6F894DEBF78
:101E00000FBECDBFDF91CF911F910F91EF90DF906B
:101E1000CF9008959091300390FF16C090911101DA
:101E200020911201921770F4E92FF0E0DF01AA0F60
:101E3000BB1FEA0FFB1FEB5CFC4F81836083428377
:101E40009F5FF0CF0C94AA0E0895CF93DF9300D03C
:101E50001F92CDB7DEB79091300390FF0AC09E016C
:101E60002F5F3F4F0E94030E4B8169818A810E9440
:101E70000A0F0F900F900F90DF91CF910895CF939D
:101E8000DF93EC01EC81F0E0E553FB4F4491E0E39C
:101E9000F3E0628181810E94250F8C818F5F8C83AA
:101EA000DF91CF910895CF93DF93EC01E0E3F3E06E
:101EB000438162818C810E94250F8C818F5F8C838E
:101EC000DF91CF9108950F931F93CF93DF9300D0AD
:101ED0001F92CDB7DEB78C018091F20181110AC04B
:101EE0009E012F5F3F4F4FEF6FEF0E94030E8A81DD
:101EF0008093F201F8018481813051F028F0823022
:101F000061F44091F2010AC08091F20140E007C003
:101F10006091F20140E080E003C040E080E060E0DA
:101F20000E940A0FF801848190E0019663E070E05E
:101F30000E94583284830F900F900F90DF91CF91C1
:101F40001F910F910895AF92BF92CF92DF92EF92BF
:101F5000FF920F931F93CF93DF9300D01F92CDB7C3
:101F6000DEB7182FF62E042FE22E9091300390FF4B
:101F70006DC0E92FE695AE2FB0E0AC58BE4F8C9106
:101F8000809347029E7F923061F49E012F5F3F4F06
:101F9000812F0E94030E4B8169818A810E940A0F62
:101FA00043C0823019F4009133033EC0863019F4E7
:101FB0001091310339C08930D9F38931A9F5E9513C
:101FC0008E2F8170D82EE695F0E0E553FA4FA5905C
:101FD000B490C12CBB2460911301C61618F52C2DAA
:101FE00030E0A29EC001A39E900DB29E900D1124E0
:101FF00070E00E944432812FD11002C0860F01C0D0
:10200000861B90911101290F311DA901440F551F05
:10201000240F351F2B5C3C4F402F6F2D0E94030E69
:10202000C394D9CF0E94AA0E10933103F0923203C9
:1020300000933303EE2051F060913003709131032F
:1020400080913203909133030E94280E0F900F90DD
:102050000F90DF91CF911F910F91FF90EF90DF9044
:10206000CF90BF90AF900895E0E3F3E09181282FE7
:102070004381628188E0890F0C94A30F81E00C9466
:102080003410E0E3F3E09181282F4381628188EFEF
:10209000890F0C94A30F81E00C944110E0E3F3E06E
:1020A000628121E1620F08F46FEF282F4381818163
:1020B0000C94A30F81E00C944E10E0E3F3E06281F6
:1020C00021E1621B08F460E0282F438181810C9498
:1020D000A30F81E00C945D10E0E3F3E0438121E184
:1020E000420F08F44FEF282F628181810C94A30FD7
:1020F00081E00C946C10E0E3F3E0438121E1421BAA
:1021000008F440E0282F628181810C94A30F81E0C4
:102110000C947B1020E00C94A30FFF920F931F935D
:10212000CF93DF93EC01F12C0FEF10E060911301DE
:10213000F616F0F4809111012F2D30E0280F311D9B
:10214000C901880F991F280F391F2B5C3C4F70E085
:10215000C8010E945832962F8C81409133036091C0
:102160003203F99E800D11240E94030EF394DECFFA
:102170000E94AA0E9A818C8190FF02C08F5F01C0DD
:1021800081508C83DF91CF911F910F91FF90089523
:10219000AF92BF92CF92DF92EF92FF920F931F9375
:1021A000CF93DF93FC01828180FF02C00FEF01C05B
:1021B00001E010E04FE0A42E80911301181708F001
:1021C00043C080911101C12ED12CE601C80FD11D51
:1021D000CE01880F991FC80FD91FCB5CDC4F198225
:1021E00018821A8234E0E32EF12CB12C8091F40194
:1021F0008B0D80312CF06A2D0E943632892F05C05C
:1022000087FF03C090911301890F082E000C990BD2
:10221000C816D90691F4809133038E9DA0018F9D3D
:10222000500D112455954795559547959E01609100
:102230003203809131030E94030EB00EF1E0EF1AD9
:10224000F108A1F61F5FB8CF0E94AA0E8091F40199
:10225000013031F4811102C080911301815007C017
:1022600090E001966091130170E00E9458328093D3
:10227000F401DF91CF911F910F91FF90EF90DF90CC
:10228000CF90BF90AF900895CF938091110190911E
:102290001201891770F4E82FF0E09F01220F331F1D
:1022A000E20FF31FEB5CFC4F1182108212828F5FF2
:1022B000F0CFC0E060911301C617C0F5EC2FF0E03D
:1022C00070E0CF010E94583220911101820F2091BD
:1022D000F301022E000C330B90E0E217F307CCF071
:1022E00020910E01022E000C330B2E173F078CF0AD
:1022F0009C01220F331F820F931F9C012B5C3C4FCC
:102300004091330360913203809131030E94030EA8
:102310000BC0FC01EE0FFF1F8E0F9F1FFC01EB5C3B
:10232000FC4F118210821282CF5FC4CF0E94AA0E8E
:1023300020910D018091F301820F8093F301909120
:102340000E01920F90930E0119165CF4082E000CEA
:10235000990B4091130150E04150510984179507A2
:102360001CF0219520930D01CF9108958F929F929B
:10237000AF92BF92CF92DF92EF92FF920F931F9393
:10238000CF93DF938C01FC014481C42FD0E09E01E8
:10239000DE010E94A3329B01AC010E94B9326B01A5
:1023A0007C01E0E2F0E0EC1BFD0BA5E5B0E09B0159
:1023B000AC010E94B9324B015C019F01DF010E9418
:1023C0009B329B01AC010E94C4329B01AC012C0DDD
:1023D0003D1D4E1D5F1DC501B4010E946C32C22F10
:1023E000D22F2A3228F4F3E02F9F900111240DC040
:1023F00025E530E02C1B3109C901880F991F280FF2
:10240000391F37FF02C02F5F3F4F35952795C22FE9
:10241000C095F12C85E5E82EED1A80911301F81690
:10242000C8F4F1FC02C08E2D01C08D2F90911101D6
:102430002F2D30E0290F311DA901440F551F240F06
:10244000351F2B5C3C4F4C2F609132030E94030ED2
:10245000F394E3CF0E94AA0EF8018481811102C097
:1024600091E003C0803219F49FEF90930C0190919A
:102470000C01890FF8018483DF91CF911F910F9197
:10248000FF90EF90DF90CF90BF90AF909F908F9094
:1024900008950F931F93CF93DF93EC0100E010E0BA
:1024A00080911301282F30E00217130724F5909133
:1024B00011019801290F311DA901440F551F240F47
:1024C000351F2B5C3C4F869590E04C81081719070F
:1024D0001CF4442331F002C0411103C04091330386
:1024E00001C040E060913203809131030E94030EED
:1024F0000F5F1F4FD5CF0E94AA0E8C8190E00196EE
:10250000817099278C83DF91CF911F910F9108954E
:102510007F928F929F92AF92BF92CF92DF92EF9273
:10252000FF920F931F93CF93DF93FC0182807480FF
:1025300081E08483EBECF4E09490EAE4F5E0E4914C
:10254000A12CF5E0BF2ECC24CA94D12CE9190E2F72
:1025500010E080911301A81608F0A2C0EA2CF12C1B
:1025600022E0281568F0BE9CF001BF9CF00D1124FC
:10257000EB50FE4F80913103808380913203818341
:1025800071100AC0BE9CF001BF9CF00D1124EB50ED
:10259000FE4F138212826AC0BE9CE001BF9CD00D28
:1025A0001124CB50DE4F8B818823F9F081508B832F
:1025B0002FEF829FC00111246C8170E00E94443291
:1025C000FB01FF27E553FB4F8491E82FE9192FEF1B
:1025D000E29FC0011124B8010E944432809133036C
:1025E000689FB00111247A8341C00E941833209162
:1025F00033032695215830E0A901440F551F322F8F
:102600002227240F351F232F33278217930774F5B2
:1026100082E0881588F40E941833B6010E9458326F
:1026200088830E941833209132032695622F70E030
:102630000E945832280F2983BE9CF001BF9CF00DE8
:102640001124EB50FE4F128280913303843120F02D
:10265000893C18F088EC01C084E1BE9CF001BF9C6D
:10266000F00D1124EB50FE4F848383838091110180
:102670009701280F311DC901880F991F280F391F95
:102680002B5C3C4FBE9CF001BF9CF00D1124EB5025
:10269000FE4F4281618180810E94030EA39459CF35
:1026A000DF91CF911F910F91FF90EF90DF90CF902E
:1026B000BF90AF909F908F907F900C94AA0EE0E314
:1026C000F3E080818E7F808360817181828193813C
:1026D0000E94280E109248022FEF80E792E02150CE
:1026E00080409040E1F700C000000C94AA0EE0E3A7
:1026F000F3E080818E7F8083109248022FEF80E785
:1027000092E0215080409040E1F700C000000C941E
:10271000AA0E60913003669570E04BE050E084E1D2
:1027200091E00E942833892B19F481E080934802BC
:102730000E944C2A90934102809340020895909108
:10274000300390FF35C09170811102C0926006C0C5
:102750008B3210F0946502C0880F982B9093300351
:10276000662351F060913003709131038091320300
:10277000909133030E94280E60913003669570E0BB
:102780004BE050E084E191E00E942833892B19F05E
:102790001092480202C00E94891381E08093430294
:1027A0004091330360913203809131030C948A107D
:1027B0000895682F90913003969581E0890F8B32B0
:1027C00008F081E00C949F1381E00C94D913682FDA
:1027D0009091300396958FEF890F09F48AE20C945B
:1027E0009F1381E00C94E71361E00C949F13E0E3E6
:1027F000F3E080818160808386950C94F41380914E
:10280000300380FD0C945F130C94F71360E00C947C
:102810009F138091460281112EC00E94C62881110B
:1028200004C00E946E290E94440E0E94240E6093F0
:1028300030037093310380933203909333036E7FA0
:1028400061F40E94440E0E94240E60933003709342
:10285000310380933203909333030E94110E109240
:1028600048028091300380FF03C086950E940614C1
:1028700081E0809346020895E0E3F3E08081816087
:10288000808386950C9406140F931F93CF93DF9348
:1028900080914802882309F495C080914702E09115
:1028A0003003E695E81BE0934202823049F4F0E001
:1028B000E953FB4FE491CE2FD0E00FE31FE059C066
:1028C000863049F4F0E0EC53FB4FE491CE2FD0E09A
:1028D00003E51FE04EC0893051F4E695F0E0EF5378
:1028E000FB4FE491CE2FD0E00DE810E142C08F30D5
:1028F00051F4E695F0E0E254FB4FE491CE2FD0E0A6
:1029000008EC10E136C0853149F4F0E0E554FB4FA6
:10291000E491CE2FD0E004E411E12BC08831D9F04E
:10292000833239F4E9EBF4E0C591D49103E61FE07A
:1029300020C08432A9F08532C1F48E2F63E00E945A
:102940002A32E92FF0E0EA54FB4FE491CE2FD0E099
:1029500008E812E10EC0C8E2D0E006EB11E109C0C0
:10296000C4EFD1E009E412E104C0C0EDD7E00FEFFD
:102970001DE080914302882361F0109243020E947F
:102980004C2A90934102809340021092450210928B
:1029900044020E944C2AE0914002F09141028E1BB9
:1029A0009F0B8F3F9F4770F4EC0FFD1FF093410288
:1029B000E093400280E492E0F801DF91CF911F9113
:1029C0000F910994DF91CF911F910F910895882362
:1029D00011F0FA0101C0FB010994CF93DF93C82FD6
:1029E000D62F0E94530E8C1740F00E94530E8D1765
:1029F00020F4DF91CF910C94E4138C2FDF91CF91D1
:102A00000C94F4131F93CF93DF93FB0112811123D6
:102A100009F4C1C0EC010E94FF278272CC3CFCE5A6
:102A2000DF0709F49BC008F043C0C63CECE5DE07B5
:102A300009F480C0D8F4C33C9CE5D90709F46DC003
:102A400038F4C23CDC4509F0A7C00E94FF136BC0FC
:102A5000C43C9CE5D90709F468C0C53CDC4509F0D5
:102A60009BC04BE450E16EE370E15BC0C93CFCE508
:102A7000DF0709F469C070F4C73CECE5DE0709F430
:102A80005EC0C83CDC4509F087C04AE550E169E614
:102A900070E147C0CA3C9CE5D90709F45AC0CB3C59
:102AA000DC4509F079C046E85EE06FE67EE039C0BB
:102AB000C13DFCE5DF0709F45EC098F4CE3C9CE51F
:102AC000D90709F452C008F44EC0CF3CFCE5DF073B
:102AD00009F44EC0C03DDC4509F05EC06EE089E0FF
:102AE00057C0C43D9CE5D90709F44BC058F4C23D1A
:102AF000FCE5DF0709F442C0C33DDC4509F04CC0EA
:102B000088E143C0C53D9CE5D907F1F1CD35DD45F0
:102B100009F042C06AE285E23BC041EF53E164EE56
:102B200073E10E94E71410E037C044EE53E161EF17
:102B300073E1F7CF4EE350E16BE470E1F2CF49E689
:102B400050E16AE570E1EDCF47E850E168E770E1F8
:102B5000E8CF48E750E167E870E1E3CF4FE65EE099
:102B600066E87EE0DECF81E010C065E082E010C064
:102B700068E086E00DC064E18FE00AC067E185E1AE
:102B800007C062E289E104C083E20E94F413CBCF64
:102B90000E94ED14C8CF11E0812FDF91CF911F91DA
:102BA00008956E9A2EB12F7B3EB130644FB7F894E2
:102BB000FC01CB01880F991F680F791F6E0F7F1FD3
:102BC000E617F70789F0819198E03EB9000000C050
:102BD00087FF2EB9880F000000C000C000C02EB9CA
:102BE00000C09A9591F7ECCF4FBF8FE594E0019725
:102BF000F1F700C00000089583E290E00E943533B1
:102C0000813281F484E290E00E943533873051F4C0
:102C100085E290E00E94353391E0833109F090E045
:102C2000892F01C080E081700895CF93C82F811152
:102C300002C06FEF01C061E283E290E00E9449337D
:102C4000C11102C06FEF01C067E084E290E00E9412
:102C50004933C11102C06FEF01C063E185E290E02A
:102C6000CF910C94493380E00E9415160C94C02833
:102C7000089586E290E00E943533682F70E080E08E
:102C800090E0089586E290E00C9449330E94381653
:102C90000E94FC1581110CC060E070E0CB010E9425
:102CA00042160E94E5170E94C41881E00C94151684
:102CB0000895CF93FB01C281CC23E9F09C012251FE
:102CC0003F452031310520F482510E94D4180CC0B8
:102CD0008031FFE59F0751F481E00E94682643E0C0
:102CE00062E081E00E949C06C0E018C081319F45EF
:102CF000A9F482E0F2CF8031EFE59E0711F481E084
:102D000004C081319F4549F482E00E94892643E056
:102D100062E081E00E949C0601C0C1E08C2FCF914F
:102D200008952FEFFC0120830895CF93DF93EC01EA
:102D30008881813889F028F48038A1F40E94A40E9B
:102D400010C0823861F0833869F40E949E0E898336
:102D50000E94A10E8A8306C00E94530E02C00E94E8
:102D6000890E8983DF91CF910895CF93DF93EC0192
:102D700088818138B1F058F4803851F5D9810E94AA
:102D8000A10EC82F0E949E0E4D2F6C2F1DC08238A1
:102D9000B1F08338E9F40E94A40E482F6A8189813A
:102DA00013C089810E9406148981811104C0DF91BA
:102DB000CF910C947713DF91CF910C943C148981BF
:102DC000DF91CF910C949B0EDF91CF910C948A10E0
:102DD000DF91CF910895EF92FF920F931F93CF93BE
:102DE000DF93EC01E62E0196E8814E2F50E0FA01C8
:102DF0003197E331F10508F09BC0E05AFF4F0C9486
:102E00008E32198289E057C08981823039F083304F
:102E100061F0813031F50E94582A02C00E943916B3
:102E20009A838B837C836D8385C08E01F12C8F2DDB
:102E30000E94570AF801828373836483F3940D5FC1
:102E40001F4FF5E0FF12F3CF75C08981823049F43E
:102E50006A817B818C819D810E9494320E944216FE
:102E600069C06E2DCE010E94911664C04B816A81AB
:102E700089810E94B7179C838D835CC02C813D8122
:102E80003227232732274B816A8189810E94D017FC
:102E900051C00E94E5174EC00E94B5164BC00E945B
:102EA000951648C00E943A0E45C00E94771824C06B
:102EB0000E94791899838A833DC06B8170E0898173
:102EC0009A81AE014C5F5F4F9827892798270E940F
:102ED0007C1830C06B8170E089819A81AE014C5FB3
:102EE0005F4F9827892798270E94A11823C00E9426
:102EF000C41820C00E94A41789831CC06B8170E095
:102F000089819A81AE014C5F5F4F98278927982766
:102F10000E9424180FC06B8170E089819A81AE01F4
:102F20004C5F5F4F9827892798270E94481802C056
:102F30008FEF88836E2DCE01DF91CF911F910F917E
:102F4000FF90EF900C944A2B84E0089550E0440FDA
:102F5000551F24E2629F400D511D11249A0164EB1C
:102F6000869F200D311D1124C901879608950F9366
:102F70001F93CF93DF930E94A6178C010E943533D5
:102F8000C82FD0E0DC2FCC27C80101960E94353332
:102F90009E01282BC901DF91CF911F910F910895B8
:102FA0000F931F93CF93DF93122F032F0E94A61727
:102FB000EC01602F0E944933612FCE010196DF9111
:102FC000CF911F910F910C944933AF92BF92CF9242
:102FD000DF92EF92FF920F931F93CF93DF93A12C79
:102FE000E12CF12CB12C00E010E0C0E0D0E0670152
:102FF000C00ED11EFE01EE0FFF1FEC0DFD1DEA5CA1
:10300000FE4F259134914C2F6B2D8A2D0E94D017A5
:103010002196C231D10571F70C5D1F4FB39485E045
:10302000B812E3CF84EBE80EF11CA39484E0A8125D
:10303000D9CFDF91CF911F910F91FF90EF90DF904B
:10304000CF90BF90AF900895EF92FF920F931F9390
:10305000CF93DF93EA017A01E60EF71E8C01C801D7
:103060008796CE15DF0569F0003D22E0120720F4B7
:103070000E943533888301C0188221960F5F1F4F4D
:10308000EECFDF91CF911F910F91FF90EF900895B8
:10309000EF92FF920F931F93CF93DF93EA017A0190
:1030A000E60EF71E8C01C8018796CE15DF0559F094
:1030B000003D22E0120718F468810E9449332196EE
:1030C0000F5F1F4FF0CFDF91CF911F910F91FF90B6
:1030D000EF900895462F843038F4753028F462312B
:1030E00018F4672F0C94B71780E090E0089580E102
:1030F000089589E091E00895EF92FF920F931F9356
:10310000CF93DF93EA017A01E60EF71E8C01C80126
:1031100089509D4FCE15DF0569F0093021E0120777
:1031200020F40E943533888301C0188221960F5FF6
:103130001F4FEDCFDF91CF911F910F91FF90EF9037
:103140000895EF92FF920F931F93CF93DF93EA01BD
:103150007A01E60EF71E8C01C80189509D4FCE15ED
:10316000DF0559F0093021E0120718F468810E9448
:10317000493321960F5F1F4FEFCFDF91CF911F9102
:103180000F91FF90EF900895CF93DF93C7EFD2E0B8
:1031900060E0CE010E9449332196C11584E0D80732
:1031A000B9F7DF91CF910895DF92EF92FF920F93DD
:1031B0001F93CF93DF9300D000D0CDB7DEB7F82EAA
:1031C0008FE08F15E8F18FEF93E00E943533811186
:1031D00037C007EF12E0FF2069F0011584E01807FF
:1031E00079F1C8010E943533811101C0FA940F5F53
:1031F0001F4FF1CF19821A821B821C82DD24D394C7
:1032000078018FEFE81AF80AC8010E9435338983E4
:103210001A828823A9F09FEF980F933058F48A837D
:10322000D9820E5F1F4FC7010E9435338B838823DD
:1032300039F07801CE0101960E94F5078701E0CFB1
:103240000F900F900F900F90DF91CF911F910F91E2
:10325000FF90EF90DF9008950F931F93CF93DF932C
:10326000C42FD22FFC0182818823C9F040934B02E6
:103270000E944C2A90934A028093490280E28C0F6C
:10328000883008F057C0C77081E001C0880FCA9528
:10329000EAF7DF91CF911F910F910C94851F8091D8
:1032A0004B02481330C08091490290914A020E941B
:1032B000642A883C910538F510E21D0FCD17B9F04E
:1032C00080E28C0F883040F4C77081E001C0880F25
:1032D000CA95EAF70E948C1F183028F581E09D2FCF
:1032E000977001C0880F9A95EAF70E94851F802F7A
:1032F0000E947C1F1830F0F4D77081E001C0880F65
:10330000DA95EAF70AC080E28C0F883098F4C7702B
:1033100081E001C0880FCA95EAF7DF91CF911F9134
:103320000F910C948C1F802FDF91CF911F910F91E3
:103330000C947C1FDF91CF911F910F9108950F93F3
:103340009C01CB01233F4CE5340731F188F4283D43
:10335000FCE53F07D9F0293D4CE5340779F1273DDD
:103360003C45A9F506E221EE41EE67ED7CE52BC078
:10337000253FFCE53F07E1F0A8F0263F3C4539F545
:1033800007E225EE46EE66EF7CE51DC007E225EE7E
:1033900045EE68ED7CE517C006E221EE40EE63EFF6
:1033A0007CE511C007E225EE44EE64EF7CE50BC03E
:1033B00006E221EE42EE65EF7CE505C008E221E081
:1033C00045EE69ED7CE50E942C1980E008C0FC0107
:1033D0008281882319F010924B0201C081E00F9185
:1033E0000895CF93DF93EC01FB018281882309F4D8
:1033F0001FC1C230FCE5DF0708F41BC1C6319CE5E4
:10340000D90738F09E012A5F3C452930310508F084
:1034100010C10E94D9289093070380930603C031FE
:10342000ECE5DE0709F4C3C008F041C0C8308CE504
:10343000D80709F49AC0F0F4C430ECE5DE0709F4CB
:1034400087C068F4C2308CE5D80709F477C0C33070
:10345000DC4509F0E3C080910603826076C0C63087
:10346000ECE5DE0709F46EC008F07BC0809106032E
:1034700088606BC0CC308CE5D80709F485C068F44F
:10348000CA30ECE5DE0709F474C008F079C00E9488
:10349000122280910603806858C0CE308CE5D80790
:1034A00009F476C008F07FC0809106038BC0CB3F43
:1034B000ECE5DE0709F44FC018F5C3318CE5D807F9
:1034C00009F47DC078F4C131ECE5DE0709F473C07E
:1034D000C231DC4509F0A2C00E941222809106038D
:1034E0008F7733C0C5318CE5D80709F472C008F472
:1034F00086C0CA3FDC4509F091C0809107033EC0F9
:10350000CF3FFCE5DF0709F45FC058F4CD3F9CE5F1
:10351000D90709F444C008F43FC0809107038260D2
:103520002DC0C130FDE5DF0709F475C008F45DC0AA
:10353000C230DD4509F072C080E06EC080910603A4
:10354000816003C08091060380618093060366C09A
:103550008091060311C08091070382608093070366
:103560005DC0809106038062F0CF80910603806485
:10357000ECCF8091060388608460E7CF8160EECF56
:10358000809106038E7FE1CF809106038D7FDDCF92
:1035900080910603877FD9CF8091070318C080915F
:1035A00007038D7FDBCF809106038F7ECECF809186
:1035B00006038F7DCACF809106038F7BC6CF809193
:1035C0000603877F8B7FC1CF809107038D7F8E7F1E
:1035D000C5CF8091060382FB222720F991E0922734
:1035E00090FB82F990FB83F9B0CF80910703982F6D
:1035F000909591708E7F892B90FB81F9AFCF0E94BF
:1036000012228091060387FB222720F991E092275E
:1036100090FB87F99ACF81E00E9470298091060380
:10362000909107030E94EA280E94122280E001C0C4
:1036300081E0DF91CF910895CF93DF9386319C4550
:1036400041F5EB010E94FF27982F8A8120911F01ED
:1036500030912001882379F09A7A81E009F480E0A2
:1036600080934C02911102C069E201C065E3C90177
:103670000E94B7290AC080914C02811102C069E200
:1036800001C065E3C9010E94B9290E94512880E068
:1036900001C081E0DF91CF9108951092B9008CE0D4
:1036A0008093B8000895EF92FF920F931F93CF93EA
:1036B000DF93182FEB011092BC0084EA8093BC00CA
:1036C0000E944C2A7C018091BC0087FD0EC0CF3F38
:1036D0008FEFD807C1F30E944C2A8E199F098C17CF
:1036E0009D0788F38EEF9FEF2EC08091B900887FF1
:1036F000883041F08091B900887F803119F08FEFD8
:103700009FEF21C01093BB0084E88093BC000E940F
:103710004C2A8C018091BC0087FD0CC0CF3F8FEFFD
:10372000D807C1F30E944C2A801B910B8C179D0770
:1037300088F3D8CF8091B900887F883111F0803428
:10374000F1F680E090E0DF91CF911F910F91FF9013
:10375000EF9008950F931F93CF93DF93EB01809326
:10376000BB0084E88093BC000E944C2A8C018091AD
:10377000BC0087FD0EC0CF3F8FEFD807C1F30E947A
:103780004C2A801B910B8C179D0788F38EEF9FEFBF
:103790000CC02091B900287F81E090E0283211F41C
:1037A00080E090E0919581959109DF91CF911F91F3
:1037B0000F9108950F931F93CF93DF93EC0184EC47
:1037C0008093BC000E944C2A8C018091BC0087FD34
:1037D0000EC0CF3F8FEFD807C1F30E944C2A801B49
:1037E000910B8C179D0788F38EEF9FEF03C080919C
:1037F000BB0090E0DF91CF911F910F9108950F933F
:103800001F93CF93DF93EC0184E88093BC000E9468
:103810004C2A8C018091BC0087FD0EC0CF3F8FEFFA
:10382000D807C1F30E944C2A801B910B8C179D076F
:1038300088F38EEF9FEF03C08091BB0090E0DF9193
:10384000CF911F910F910895CF92DF92EF92FF9247
:103850000F931F93CF93DF93C62F6A017901B801AD
:103860000E94531B97FD11C0B8018C2F0E94AA1B08
:10387000E601EC0CFD1CCE15DF0539F097FD05C007
:10388000B80189910E94AA1BF6CF24E92093BC00BD
:10389000DF91CF911F910F91FF90EF90DF90CF902C
:1038A0000895CF92DF92EF92FF920F931F93CF93E1
:1038B000DF93D82EC62E7A01E901B8010E94531B6E
:1038C00097FD2AC0B8018C2D0E94AA1B97FD24C029
:1038D000B8018D2D81600E94531B670121979601CD
:1038E0002E193F092C173D0768F497FD15C0C80134
:1038F0000E94DA1B97FD02C0F6018083FFEFCF1A0A
:10390000DF0AEDCF97FD08C0C8010E94FF1B97FD9D
:1039100003C0CE0DDF1D888324E92093BC00181658
:10392000190614F480E090E0DF91CF911F910F9180
:10393000FF90EF90DF90CF90089590935202809384
:1039400051020895E0915102F0915202309721F016
:103950000190F081E02D099480E00895E0915102FA
:10396000F0915202309721F00280F381E02D09940A
:103970000895E0915102F0915202309739F022E01F
:10398000DC012C930480F581E02D099408952091A9
:103990004F02309150022817390771F0909350026E
:1039A00080934F02E0915102F0915202309721F042
:1039B0000680F781E02D0994089520914D02309101
:1039C0004E022817390771F090934E0280934D02F2
:1039D000E0915102F0915202309721F00084F1857C
:1039E000E02D099408950E94582A60936C02709308
:1039F0006D0280936E0290936F02609368027093E1
:103A0000690280936A0290936B02089585B780687B
:103A100085BF85B7806885BF089581E008950C94BF
:103A20000D1D08950C94111D0C94111D0C94141D62
:103A30000C94111D0C94181D0C94111D0E94061D50
:103A40008EEB98E20E94BD2A0E941C1D0C941A1D48
:103A50000E94121D0C94111D0E94432A0E94710A9B
:103A60000E9446160E9409140C94161D2F923F9234
:103A70004F925F926F927F928F929F92AF92BF927E
:103A8000CF92DF92EF92FF920F931F93CF93DF932A
:103A9000CDB7DEB72C970FB6F894DEBF0FBECDBF03
:103AA0000E94880A81110E94F31C84E592E09C87A1
:103AB0008B8700E010E0302E802F0E94570A2B01E8
:103AC0003C01EB85FC8581919191A191B191FC879D
:103AD000EB875301420188269926AA26BB2681142A
:103AE0009104A104B104B1F40F5F1F4F053011051B
:103AF00011F78FEF89838A831B820E944C2A816091
:103B0000782F9D838C8349815A816B818D810E949E
:103B1000191E4EC08091FA0281FD0E94630A212C79
:103B2000C12CD12C7601C394D501C4018C219D21D7
:103B3000AE21BF21892B8A2B8B2B89F10E940F1D6F
:103B40008823C9F02E823F824C205D206E207F208A
:103B500081E045284628472809F480E088870E94AC
:103B60004C2A8160782F9A8789874E815F8168858A
:103B70008A850E94191E000F111F000F111FF801E6
:103B8000EC5AFD4F80819181A281B381C826D9264C
:103B9000EA26FB26C082D182E282F38209C0239406
:103BA000CC0CDD1CEE1CFF1CF2E12F12BDCF9CCF14
:103BB0000E9444140E944A0C0E94A21C909153023D
:103BC0008917F1F00E94A21C809353022C960FB625
:103BD000F894DEBF0FBECDBFDF91CF911F910F9143
:103BE000FF90EF90DF90CF90BF90AF909F908F901D
:103BF0007F906F905F904F903F902F900C9414089F
:103C00002C960FB6F894DEBF0FBECDBFDF91CF91DB
:103C10001F910F91FF90EF90DF90CF90BF90AF90EA
:103C20009F908F907F906F905F904F903F902F90DC
:103C30000895DF92EF92FF920F931F93CF93DF933C
:103C4000CDB7DEB72B970FB6F894DEBF0FBECDBF52
:103C5000F42E052F162FE72ED82E61110E941F2853
:103C6000FE01319686E0DF011D928A95E9F77E2DEF
:103C70004F2D502F612F8D2D9E810E94CB242B968E
:103C80000FB6F894DEBF0FBECDBFDF91CF911F916D
:103C90000F91FF90EF90DF900895FC01808191815A
:103CA0000E949F270895CF93882309F4A4C0C82FAA
:103CB0008238C1F40E94A21C81FD9DC069E38091FD
:103CC0001F01909120010E94B7290E9451282FEFD7
:103CD00081EE94E0215080409040E1F700C0000068
:103CE00069E319C0833801F50E94A21C80FD83C0DE
:103CF00063E580911F01909120010E94B7290E94E5
:103D000051282FEF81EE94E0215080409040E1F760
:103D100000C0000063E580911F01909120010E9486
:103D2000B929CF910C9451288438C1F40E94A21C67
:103D300082FD61C067E480911F01909120010E9483
:103D4000B7290E9451282FEF81EE94E02150804046
:103D50009040E1F700C0000067E4DDCF8CEF8C0FEE
:103D6000813AD0F46C2F80911F01909120010E9424
:103D70008129882349F06C2F80911F0190912001A7
:103D80000E94B9290E9451286C2F80911F019091A7
:103D900020010E94B729C5CF80E28C0F883048F4FB
:103DA000C77081E001C0880FCA95EAF70E94022817
:103DB000B8CFEBE5EC0FE33040F4F0E0E353FE4F17
:103DC000808190E0CF910C94C71CE8E5EC0FE731BF
:103DD00050F4F0E0EE0FFF1FE156FE4F808191811D
:103DE000CF910C94DD1CC03F30F08C2F0E945A0BF9
:103DF000CF910C942C0CCF910895882309F464C0C2
:103E0000823879F40E94A21C81FF5EC069E3809130
:103E10001F01909120010E94B7290E94512869E357
:103E200010C08338B1F40E94A21C80FF4DC063E52E
:103E300080911F01909120010E94B7290E94512872
:103E400063E580911F01909120010E94B9290C9493
:103E50005128843879F40E94A21C82FF35C067E49F
:103E600080911F01909120010E94B7290E94512842
:103E700067E4E7CF9CEF980F913A10F4682FE1CFF9
